:0600000000308A005128C7
:10000800F90003088301C7000A08C8008A017A08B2
:10001800CB0083010C1C4828DE308E003C308F005A
:100028000C10A20A0319A30A2308803AFA008030A8
:100038007A02053003192202031C3228A201A30107
:10004800201C28288714292887100310A00C211C9D
:100058002F280714302807100310A10C270826049E
:1000680003193C28A6080319A703A60305163D286B
:1000780005122508240403194728A4080319A50311
:10008800A4038516482885124B08FA0048088A00F8
:1000980047088300F90E790E0900203084003D30AE
:1000A80068200030CA008E30C9003D3084004730D7
:1000B8006D200317A001A101A201A30183018A11E8
:1000C800C02904068001840A0406031D652864000B
:1000D8000034FA008A117B208A118000840A0408FF
:1000E8007A06031900346E2883120313C900CA1B49
:1000F80086284A1B8E284A088A004908C90A031913
:10010800CA0A820083134A1883174908C90A840057
:1001180000080800D23400345134013490340134DA
:1001280035340234583402348301BC0081389F00CE
:100138009F149F189D281E080317A10083160313F8
:100148001E0883120317A0002108FB002008FA00EC
:10015800031308008B13083098207A08BA007B082C
:10016800BB008B1764003E083B02031DBD283D08F9
:100178003A020318C228FA01FB01080040083B02B2
:10018800031DC8283F083A020318CE280130FA0098
:10019800FB01080042083B02031DD42841083A022B
:1001A8000318DA280230FA00FB01080044083B0271
:1001B800031DE02843083A020318E6280330FA0032
:1001C800FB01080046083B02031DEC2845083A02DB
:1001D8000318F2280430FA00FB0108000530FA0081
:1001E800FB01080005308301AC004829AD01AE20B1
:1001F8002D082D072E3E840083137A088000840A78
:100208007B088000AD0A06302D02031CFB28640021
:10021800303084002E080006031D15292F08840A93
:100228000006031D4829323084002E080006031DED
:1002380020292F08840A0006031D48293430840029
:100248002E080006031D2B292F08840A0006031D0B
:100258004829363084002E080006031D36292F0849
:10026800840A0006031D4829383084002E08000639
:10027800031D41292F08840A0006031D48292F0859
:10028800FB002E08FA000800AC032C0FFA282F08F0
:10029800FB002E08FA0008008301AC01AD018710AD
:1002A8000714FA30FC00FD012D08FB002C08FA00A9
:1002B8008A11CD228A117E08AE007F08AF00803AED
:1002C800FA0080307A02013003192E02031C7429C7
:1002D80000000000AE080319AF03AE032F0863291E
:1002E80087140710FA30FC00FD012D08FB002C08CC
:1002F800FA008A11CD228A117E08AE007F08AF006D
:10030800803AFA0080307A02013003192E02031C69
:10031800952900000000AE080319AF03AE032F08AB
:1003280084296400AC0A0319AD0A2D08803AFA0042
:1003380080307A02323003192C020318080053293E
:1003480004308316031391000730831299000F308D
:10035800831685003C30870010309F003C308312A4
:100368008F00AF308E000C109010101483160C14F0
:1003780083128710071008007130831603138F004B
:10038800A42105128512502187100710AA01AB017C
:10039800F6207A08A8007B08A90028040319D9299F
:1003A8002808053A2904031DDC290230AA00AB01FC
:1003B80028032904031DE229AA01AB018B170B1797
:1003C80064008719EC29A008031DEC29CC30A00093
:1003D8000719F329A008031DF329AA30A000F62065
:1003E8007A08A8007B08A900640028040319012AD8
:1003F8002808053A2904031D062A0230AA00AB0181
:10040800FF30A1002B082A04031D212A2808023ADC
:100418002904031D122A0330AA00AB012808033A55
:100428002904031D1A2A0430AA00AB012808043A3B
:100438002904031D9D2A05309B2A2A08033A2B0408
:10044800031D2D2A2808043A2904031D462A0530CD
:10045800442A2A08043A2B04031D392A2808043A96
:100468002904031D5A2A0630582A2A08053A2B045B
:10047800031D4D2A2808023A2904031D462A033081
:10048800AA00AB012808033A2904031D622A073091
:10049800602A2A08063A2B04031D682A2808033A0A
:1004A8002904031D5A2A0430AA00AB012808023A7D
:1004B8002904031D622A0830AA00AB012803290475
:1004C800031D9D2AAA019C2A2A08073A2B04031D0A
:1004D800822A2808043A2904031D752A0530AA002F
:1004E800AB012808023A2904031D7C2AAA01AB01A2
:1004F80028032904031D9D2A09309B2A2A08083A43
:100508002B04031D9D2A2808043A2904031D8F2A59
:100518000630AA00AB012808033A2904031D962ACD
:10052800AA01AB0128032904031D9D2A0A30AA0049
:10053800AB012A08093A2B04031DAC2AA108031DA4
:10054800A72AAA30A1000430A600A701AA01AB017E
:100558002A080A3A2B04031DBB2AA108031DB62A40
:10056800CC30A1000430A400A501AA01AB012A08DF
:10057800023A2B040319C42A2A032B04031DE42975
:1005880028032904031DCA2AAA01AB01AA01AB0149
:10059800E429FE01FF010310FD0CFC0C031CDB2AFF
:1005A8007A08FE077B0803187B0AFF070310FA0D79
:0C05B800FB0D7C087D0403190034CF2AE1
:02400E00EC3F85
:1042000000000000000000000000000000000000AE
:10421000000000000000000000000000000000009E
:10422000000000000000000000000000000000008E
:10423000000000000000000000000000000000007E
:10424000000000000000000000000000000000006E
:10425000000000000000000000000000000000005E
:10426000000000000000000000000000000000004E
:10427000000000000000000000000000000000003E
:10428000000000000000000000000000000000002E
:10429000000000000000000000000000000000001E
:1042A000000000000000000000000000000000000E
:1042B00000000000000000000000000000000000FE
:1042C00000000000000000000000000000000000EE
:1042D00000000000000000000000000000000000DE
:1042E00000000000000000000000000000000000CE
:00000001FF
